:1000000085EF00F0EA6A0D0EE96EEF500EE01F0E6C
:10001000016E006A002EFED7012EFBD71F0E006E68
:10002000002EFED70000EF2EF2D7B5EF00F0010E44
:100030000D5E0CE3EA6A0D0EE96EEF5007E0060E66
:10004000006E002EFED700D0EF2EF9D7000CFF0E69
:10005000936E81CF05F0076A05C000F00A50016E6B
:1000600004E0D8900032012EFCD700A002D00A0E86
:10007000076E0A501A0DF3CF08F007500824946A4F
:100080008B6E0CC00DF0D3DF928880B805D00B2C9E
:1000900003D00B6A929A899A928880A80DD00B524D
:1000A0000BE1010E0B6E0A2A04500A5C03E10A6A96
:1000B000080E086E929A898ACFEF00F0946A8B6AD4
:1000C0000CC00DF0B4DF080E086EFF0E936E81CFEA
:1000D00005F0929A898A066A0450065C12E2076A61
:1000E00005A002D00A0E076ED890053207500824EA
:1000F000946A8B6E0CC00DF09ADF1A0E0826062A41
:10010000EBD7929A899AD3EF00F0F86AD09EEA6A08
:10011000E96A7E50E00B7E6EC198C19A000E7F6E38
:10012000799A79987B6A7A6A7E50E00B7E6EC198E4
:10013000C19A000E7F6EC290C69A949A9488949643
:10014000010EC66E000EC76ED190800ED56ECD6AC0
:10015000000ECA6E000ECB6EB16A799A7998040EC1
:100160007B6E7A6E0A0E0D6E4DD7000E946E929ACB
:10017000066A096A0A6A928280B203D0080E046E87
:1001800002D0040E046E928680B603D0020E0C6E6E
:1001900002D00A0E0C6E928480B401D058D792849B
:0A01A00080A401D08BD7E7D703003D
:020000040030CA
:0E00000000C6190E000F81000FC00FE00F4068
:00000001FF
